:100000000C9435020C9452020C9452020C9452023D
:100010000C9452020C9452020C9452020C94520210
:100020000C9452020C9452020C9404260C94D82680
:100030000C94E8200C9452020C9452020C9452023C
:100040000C9452020C9452020C9452020C945202E0
:100050000C9452020C946F210C9452020C94520294
:100060000C9452020C9452020C9452020C945202C0
:100070000C9452020C9452020C9452020C945202B0
:100080000C9452020C9452020C9452020C945202A0
:100090000C9452020C9452020C9452020C94520290
:1000A0000C9452020C9452020C94520200570250CB
:1000B0000600C35C01570357AC00AB00AE00AD00B7
:1000C0000357025714001500520704571D011C0165
:1000D00013000A0000047F3F1F6432146432147856
:1000E0003C1E1E140A052223252628292A2C2D2FE2
:1000F0003032333536383A3B3D3E4042434547493E
:100100004A4C4E5051535557595A5C5E6062646672
:1001100068696B6D6F71737577797B7D7F8183857E
:1001200087898A8C8E90929496989A9C9E9FA1A380
:10013000A5A7A8AAACAEAFB1B3B4B6B8B9BBBCBEA4
:10014000BFC1C2C3C5C6C7C9CACBCCCDCED0D1D220
:10015000D2D3D4D5D6D7D7D8D9D9DADADBDBDBDC22
:10016000DCDCDCDCDDDDDDDDDCDCDCDCDCDBDBDBCE
:10017000DADAD9D9D8D7D7D6D5D4D3D2D2D1D0CE2E
:10018000CDCCCBCAC9C7C6C5C3C2C1BFBEBCBBB933
:10019000B8B6B4B3B1AFAEACAAA8A7A5A3A19F9EB1
:1001A0009C9A98969492908E8C8A89878583817F79
:1001B0007D7B79777573716F6D6B6968666462605A
:1001C0005E5C5A5957555351504E4C4A4947454326
:1001D00042403E3D3B3A3836353332302F2D2C2AC3
:1001E000292826252322FFAA7F554000010101016D
:1001F00001010101010202020202020202020303E2
:1002000003030303030304040404040404050505B1
:100210000505060606060607070707070808080873
:10022000090909090A0A0A0B0B0B0C0C0C0D0D0D20
:100230000E0E0E0F0F0F10101111111212131314B6
:1002400014151516161717181819191A1A1B1B1C2E
:100250001D1D1E1E1F202021222223242425262688
:10026000272829292A2B2C2D2D2E2F3031323233BD
:100270003435363738393A3B3C3D3E3F40414243C6
:100280004445464748494A4C4D4E4F5051535455AA
:100290005658595A5B5D5E5F616264656668696B5A
:1002A0006C6D6F7072737577787A7B7D7E808283D8
:1002B0008587888A8C8E8F91939596989A9C9EA01C
:1002C000A2A3A5A7A9ABADAFB1B3B5B7BABCBEC029
:1002D000C2C4C6C9CBCDCFD1D4D6D8DBDDDFE2E4F2
:1002E000E7E9EBEEF0F3F5F8FAFDFF16036D0069B0
:1002F000006E0069004D004100430052004F003580
:100300000000001E036C006500610066006300755C
:100310000074007400650072006C0061006200737C
:100320000000000403090409023B00020100A0FAD6
:10033000090400000103010100092111010001224B
:1003400040000705810308000109040100010300C2
:10035000000009211101000122B6000705820320D7
:1003600000011201000200000008EBCE07000100AE
:100370000102000105010902A10185020901A10094
:100380000509190129081500250195087501810243
:100390000501093009311581257F9502750881060F
:1003A00009381581257F950175088106050C0A38E5
:1003B000021581257F950175088106C0C0050109D8
:1003C00080A101850319012AB700150126B7009500
:1003D0000175108100C0050C0901A10185041901F6
:1003E0002AA002150126A002950175108100C00502
:1003F000010906A1018506050719E029E715002571
:10040000019508750181020507190029EF150025DE
:100410000195F075018102050819012905950575F9
:10042000019102950175039101C005010906A10121
:10043000050719E029E715002501950875018102D6
:100440009501750881010507190029FF150026FF90
:10045000009506750881000508190129059505759F
:10046000019102950175039101C011241FBECFEFC8
:10047000DAE0DEBFCDBF12E0A0E0B1E0E8EAF3E5EC
:1004800002C005900D92A033B107D9F723E0A0E395
:10049000B2E001C01D92A635B207E1F70E946511D6
:1004A0000C94BC290C940000CF93C62F811114C06A
:1004B00080913C0290913D020E94F403813031F022
:1004C000882321F0823011F0833049F089EAC1118C
:1004D00001C08AEA0E941E0581E0CF91089582E55D
:1004E000C111F8CF81E5F6CFCF93DF93EC0160E047
:1004F0000E941708882331F020E04FEF6FEF85E569
:100500000E94B61661E0CE010E941708882331F0E0
:1005100020E04FEF6FEF80E00E94B61662E0CE0160
:100520000E941708882331F020E04FEF6FEF8AEA2E
:100530000E94B61663E0CE010E941708882331F0AE
:1005400020E04FEF6FEF8FEB0E94B616CE01DF91E8
:10055000CF91089520E04FEF6FEF85E50E94B6162A
:1005600008959C013A9521153F4150F5FC01EE2775
:10057000F170BC0166277270AC01442754709C0175
:100580002227387094FF0EC080E1EF2B09F480E041
:10059000672B09F08062452B09F08064232B89F0DA
:1005A0008068089581E0EF2B09F480E0672B09F063
:1005B0008260452B09F08460232B19F08860089530
:1005C00080E00895CF93DF93EB010E94B102FE011A
:1005D0000995DF91CF910895CF93DF93EC01805E71
:1005E0009109089720F06FE677E0209711F467E211
:1005F00075E0CE010E94E2028C2F0E948804DF91F8
:10060000CF910895CF93DF93EC010E94D404CE01E3
:10061000805E9109089720F066E777E0209711F453
:100620006EE275E0CE010E94E202DF91CF91089563
:1006300081E0089581E008950E941A0308950895C5
:100640000E941F030895A5E0B0E0E9E2F3E00C94F6
:100650001D2949835A833091370289819A8131114A
:1006600019C0662399F0222389F00E94F408182FFC
:10067000682F89819A810E94D90869817A81812FA6
:100680000E946E0F2596E3E00C9439290E94E6083B
:10069000182FF3CF0E94F40869817A81F1CFFC0111
:1006A000262F408151816281738184810E942303BE
:1006B000089581E00895CF93DF93EC0160E00E94FC
:1006C0004F03BE010E942003DF91CF9108950E9445
:1006D0008F1008950E949310089508950E94930723
:1006E0000E946D032FEF84E39CE0215080409040F6
:1006F000E1F700C0000008950E946E030E9493215C
:1007000008950E946E030E94A42108950F931F93E1
:10071000CF93DF938C0161E00E944F03EC01B8019D
:100720000E94D51EB801CE010E941C03811106C093
:1007300080E0DF91CF911F910F910895B801CE0114
:100740000E94F61E8823A1F3B801CE010E94161E56
:10075000882371F3B801CE010E94221B882341F344
:10076000B801CE010E94881D882311F3B801CE0183
:100770000E942E1A8823E1F2F8018281882361F019
:10078000CB35FDE5DF0701F158F4C115ECE5DE07D7
:1007900091F0CF3DDC4591F0C8010E941803C9CF0C
:1007A000CD358DE5D80769F090F0C83ADD45A1F761
:1007B0000E948103BDCF0E947C03BACF0E94AA0D84
:1007C000F7CF0E94EF0CE8CF0E94F90CE5CF0E9412
:1007D000FD0CE2CF0E94CA200E942B0408950E94C3
:1007E0002F040E94CF200895292F332740E02115A0
:1007F000310511F0C90148E09C0164E03695279568
:100800006A95E1F72115310511F04C5FC9019C0192
:1008100036952795369527952115310511F04E5FB0
:10082000C90196958795892B09F04F5F842F08950C
:1008300008950E941804089581E008950E941C0400
:1008400008950895CF93C82F0E9419048C2F0E94F9
:100850001E04CF91089580E00E94220408950E9412
:100860007B1F0E9422040895CF930E947B1FC82FF4
:10087000809132028C1779F0C09332020E94542189
:100880006093330270933402809335029093360262
:100890008C2F0E942204CF910895ABE0B0E0E3E5F5
:1008A000F4E00C941E294F83588769877A878B87D9
:1008B00061110E943A0C1E821D8285E0FE0137966E
:1008C000DE01119601900D928A95E1F78C819D8150
:1008D000892B61F449815A816B817C818D819E8154
:1008E0000E94600B2B96E2E00C943A2989819A8150
:1008F00089238F3F79F3CE0101960E94590381111C
:10090000E9CFF0CFFC01808191810E9426090895F2
:10091000CF93C82F8823B9F08CEF8C0F813AA8F4BD
:100920006C2F80915F01909160010E94F01F8823DD
:1009300029F08C2F0E94F70B0E945B0C8C2F0E94D9
:10094000EF0B0E945B0CCF91089580E28C0F8830F2
:1009500048F4C77081E001C0880FCA95EAF70E9489
:100960001A0CEFCFEBE5EC0FE33040F4F0E0E95484
:10097000FE4F808190E00E94B01FE5CFE8E5EC0FCC
:10098000E73150F4F0E0EE0FFF1FE757FE4F808194
:1009900091810E94C61FD7CFCD3EA8F28C2F0E9416
:1009A000E9110E94BC12CFCF882379F19CEF980FF8
:1009B000913A28F40E94F70B0E945B0C089590E294
:1009C000980F983050F4877091E001C0990F8A9584
:1009D000EAF7892F0E94200CEFCF9BE5980F933008
:1009E00028F490E080E00E94B01F089598E5980FE9
:1009F000973128F490E080E00E94C61F08958D3E54
:100A000020F00E9443120E94BC1208951F93CF93BE
:100A1000DF93182FEB010E948804209739F4812F6F
:100A20000E94D404DF91CF911F9108958FE99FE038
:100A30000197F1F700C000002197EFCF70E060E070
:100A4000893311F460E570E00E940605089588235B
:100A500021F00E941A0C0E945B0C0895882321F05B
:100A60000E94200C0E945B0C0895B0E0A0E0EBE334
:100A7000F5E00C9417296C01D62FC72FFC011281C9
:100A8000F580F2949FE0F9220E94100CE82E882352
:100A9000B9F0E12E1123A1F08C2F807F803421F05A
:100AA00080E28D0F8830D0F080912E0382FF16C037
:100AB00082E00E94BE0C0E94100C91E0E82EE92614
:100AC000BC2EB2948FE0B822FBE0FB1508F468C09E
:100AD000EB2DF0E0E254F64D0C94D728E12CF0CF4A
:100AE0000C2F0F70C07F11F00295007F112399F039
:100AF000002359F080E28D0F883010F0D11107C02B
:100B0000802F0E941A0C0E945B0C8D2F41C0802FF9
:100B10000E942D0CF8CF8D2F0E94D404002309F4DD
:100B20003FC080E28D0F883010F0D11104C0802FBB
:100B30000E94200C03C0802F0E94330C0E945B0C8B
:100B40002FC00C2F0F70C07FC03211F00295007FB4
:100B5000DD2381F0D13009F463C0112309F46DC0A5
:100B6000FF2009F463C0F601858180FFCECF8F702E
:100B700085835CC080912E0382FD33C0112359F020
:100B8000002329F0802F0E941A0C0E945B0C80E049
:100B90000E94880405C080E00E94D4040111C7CFE0
:100BA000EB2DE850FF0B349720F40E947B1F0E942E
:100BB0002204EE2089F00E940C0C80FD0DC0F6018D
:100BC00012820E94060C0E943708C6010E94450747
:100BD0000E94060C0E944708CDB7DEB7E9E00C94EE
:100BE0003329112389F0F11006C00E943D0C802B9F
:100BF0000E942705D5CF21E0F212F7CF0E943D0CCD
:100C0000802B0E94440CCCCFF11006C00E94510CE6
:100C1000802F0E942E05C4CF31E0F31609F2F6CFE3
:100C2000112331F085E08F1508F4BACF802FE0CF83
:100C300094E09F1508F4B4CFEBCFFF2049F3D933EC
:100C400049F4FFEF27EE33E0F15020403040E1F768
:100C500000C000008D2F0E94D404A2CF8C2F869557
:100C60008695837069F0813009F09ACF8D2F9C2F83
:100C70009370111102C090E080E00E94C61F90CFD7
:100C80008D2F9C2F9370111102C090E080E00E9484
:100C9000B01F86CF8D2F112329F00E94E9110E94E9
:100CA000BC127ECF0E944312FACF8C2F8370A1F525
:100CB000111176CF4D2F429546954770440F440F42
:100CC0002D2F2F7030E0042E02C0220F331F0A9404
:100CD000E2F790E080E0D4FF09C08FE090E002C02E
:100CE000880F991F4A95E2F780959095C695C6950D
:100CF000C370822B932BC23049F058F4C13019F0E5
:100D00000E94F4074DCF0E94EB074ACF0E94FD07D7
:100D100047CF0E94E80744CF8695112311F08C2F0E
:100D20008170882309F43CCF4D2F4295469547703A
:100D3000440F440F2D2F2F7030E0042E02C0220FDD
:100D4000331F0A94E2F790E080E0D4FF09C08FE0FF
:100D500090E002C0880F991F4A95E2F78095909520
:100D6000C695C695C370822B932BC23049F058F4B8
:100D7000C13019F00E94720813CF0E94690810CF89
:100D80000E947B080DCF0E9409080ACFCF70112363
:100D900029F08C2F0E9437088D2F2ACF8D2F0E948B
:100DA0002E058C2F0E944708FBCED23F51F160F4F4
:100DB000D03FB9F0D13F81F0112309F449C0F110BF
:100DC000A4CE8C2F8F7121C0D33F11F1D43FA1F756
:100DD00080912E0382FD26C08C2F8F71112311F379
:100DE00014C0112349F084E08F1508F4D9CE8C2F5C
:100DF0008F710E945908D4CE95E09F1508F4D0CE8B
:100E0000F6CF8C2F8F711111CDCF0E943708C8CE2D
:100E1000112329F08C2F8F710E942B08C1CE0E94C4
:100E20001208BECE112349F0CF718C2F0E943708D3
:100E300063E08C2F0E94A00CB3CE81E00E94BE0C18
:100E4000E1E0EF1508F0ACCE82E00E94BE0CA8CE27
:100E5000F110F5CE8C2F8F71A5CF0F931F93CF93E9
:100E6000DF93EC01688179818A810E9431098C01CC
:100E70000E9484080E94E707B801CE010E94350550
:100E8000DF91CF911F910F910895CF93DF93EC01E4
:100E90008B819C81892B29F08881998189238F3FBF
:100EA00051F4DF91CF910895CE010E942D07CE011C
:100EB0000E945B03F6CFCE010E9486038111F4CF1E
:100EC0000E94100C882369F38A81882351F3809152
:100ED0002E0382FFE6CF82E00E94BE0CE2CF882381
:100EE00021F00E942D0C0E945B0C0895882321F0B4
:100EF0000E94330C0E945B0C089590E080E00E94F9
:100F0000B01F90E080E00E94C61F0E943A0C0E9431
:100F10005B0C0E94D8120E94BC1208950E94FF0B25
:100F20000E947D0708950E94270C0E948E07089555
:100F300092959F70963091F058F4925F9F70923026
:100F400058F4803F19F030F4883E30F481E0089581
:100F50009A5FF4CF843FD1F380E00895883EB0F3E8
:100F6000813FD1F7F3CFFC0183819481892B29F054
:100F70008081918189238F3F11F480E008958081E1
:100F800091810E9426090E9498070895A5E0B0E08B
:100F9000ECECF7E00C941E292596E2E00C943A293B
:100FA000A6E0B0E0E6EDF7E00C941E292696E2E01C
:100FB0000C943A2908950E94DA0708950E94DB07ED
:100FC00090933F0280933E020E947D07089508950A
:100FD0000E94DE07089520913E0230913F02822B4D
:100FE000932B0E94DE07089520913E0230913F022C
:100FF000822393230E94DE07089520913E023091C0
:101000003F02822793270E94DE0708950E94740200
:1010100008950E94060890933D0280933C020E942E
:101020007D07089590E080E00E94090808950097E8
:1010300029F481E0662371F080E00CC021E030E00B
:1010400002C0220F331F6A95E2F72823392381E07B
:10105000232B91F3089521E030E0A90102C0440F51
:10106000551F8A95E2F7CA010E940908089521E0F8
:1010700030E002C0220F331F8A95E2F780913C02D4
:1010800090913D02822B932B0E940908089521E044
:1010900030E002C0220F331F8A95E2F72095309589
:1010A00080913C0290913D02822393230E94090883
:1010B000089521E030E002C0220F331F8A95E2F745
:1010C00080913C0290913D02822793270E9409085B
:1010D000089520913C0230913D02822B932B0E9477
:1010E0000908089520913C0230913D028223932308
:1010F0000E940908089520913C0230913D02822708
:1011000093270E94090808950895262F277091E0DB
:1011100001C0990F2A95EAF723E0769567952A95FD
:10112000E1F7660F771F660F771FFA01E60FF71FCB
:1011300050E040E0682F70E08191DF0111979B0142
:10114000042E02C0369527950A94E2F72170219566
:101150002827292328272C934F5F5F4F44305105C0
:1011600059F70895A82FA77023E0969587952A959B
:10117000E1F7880F991F880F991FFB01E80FF91FEE
:1011800050E040E080E0219130E00A2E02C0369528
:1011900027950A94E2F721703327042E01C0220F0D
:1011A0000A94EAF7822B4F5F5F4F4430510559F79D
:1011B0000895262F911109C0853038F4682F70E00A
:1011C00048E352E0822F0E948508089591110AC0D9
:1011D000853030F468E372E090E00E94B208982F06
:1011E000892F089590E0FCCFB0E0A0E0EAEFF8E0AE
:1011F0000C9417297C0100913C0210913D028091D2
:101200003E0290913F02082B192BCFE0D0E0CC2476
:10121000C394D12CBC2EC6010C2E02C0880F991F7E
:101220000A94E2F780239123892B49F4219790F7C0
:10123000B12C8B2DCDB7DEB7E9E00C943329B70183
:101240008C2F0E94830F019789F3F3CFCF93DF9305
:10125000EC010E94F408BE010E94830FDF91CF9140
:1012600008951F93CF93DF93EB0190913702992359
:1012700039F0CB010E942609DF91CF911F9108958B
:10128000882369F0CB010E94F408182F682FCE0143
:101290000E94D908BE01812F0E94830FEDCFCB01A0
:1012A0000E94E608182FF6CF1F93CF93DF93C091CB
:1012B000400216E0809141028C1304C0DF91CF916F
:1012C0001F910895D0E01C9FF0011D9FF00D112487
:1012D000EE5BFD4F408151816281738184819581F4
:1012E0000E94D0072196C770E5CF409172025091BD
:1012F00073026091740270917502809176029091F0
:1013000077020E94D00708951F93CF93DF938091B7
:101310007702807F09F049C080917402882309F424
:1013200044C080914002C09141026091720270916C
:101330007302A0917502B0917602D62FD72316E0E2
:10134000C81799F190E0109711F0DF3F19F401965A
:101350008770F6CF189F9001199F300D1124F90165
:10136000EE5BFD4F41814713F2CF40814613EFCF33
:1013700042814111ECCF438154814A1B5B0B483CB5
:10138000510528F7809177028F70806180937702F2
:10139000F901E95BFD4F80818F708061808382E776
:1013A00092E00E9445070E945409DF91CF911F915E
:1013B0000895A1E1B0E0EFEDF9E00C9416298C015D
:1013C00085E0F801DE011D9601900D928A95E1F706
:1013D000F801E28082E7C82E82E0D82E6091750283
:1013E000709176026115710509F44EC190917202F7
:1013F00020917302892F82238F3F09F445C14081D8
:101400005181A380B480F0907402F501E61BF70BC4
:10141000FF2009F4EAC080917702382F307FE83C42
:10142000F10508F0A3C031116DC0FE2C251316C0C4
:10143000941314C0E11012C08F7080618093770202
:101440000E947509C6010E94450780917702F80144
:1014500085838F2D6196EAE00C943229A114B104A2
:1014600029F0842F85238F3F09F027C180E0F82FD2
:10147000F170DF2E80FF3CC080914002209141023C
:1014800036E0821315C04D875E878D859E850E944C
:101490002609292F22952F702230F0F0243018F5DC
:1014A0009F70F1F0F8019581907FD1F4D12C1EC08E
:1014B00090E0389FF001399FF00D1124EE5BFD4F55
:1014C0006181651306C06081641303C06281E61206
:1014D0000FC001968770D5CF9F7011F0882331F32C
:1014E000805E883018F3C8010E944507FD2CB1CFFB
:1014F000EE2009F4AECF809177028160809377026D
:10150000F12CA7CF251306C0941304C0F801EE20D8
:1015100009F487C0C8010E94B307882319F1EE209F
:1015200009F180917702803270F02091720230913F
:10153000730238872F831986BB86AA868C87CE01D3
:1015400007960E94450786E0F801A2E7B2E0019005
:101550000D928A95E1F70E9484090E947509FF2483
:10156000F39477CFC8010E944507F9CF311113C01A
:101570007A2DB98AA88A6E2D89890E94C60782E7CA
:1015800092E00E94450786E0F60111928A95E9F7FC
:101590000E947509B5CF25130FC094130DC0E1103B
:1015A0000BC0F8018583C8010E94450786E0F6015B
:1015B00011928A95E9F74DCFC8010E94B30788239D
:1015C00089F2EE2079F280917702803208F4BBCF65
:1015D00020917202309173023A8329831B82BD826B
:1015E000AC828E83CE010196ACCFE83CF10508F0C9
:1015F0003EC0FE2CEE2009F4B5CF25132AC094136B
:1016000028C08091770280FD1BC0982F907FC1F089
:10161000F8018583903F31F0982F907F905F8F7015
:10162000892B8583C8010E94450786E0F801A2E75F
:10163000B2E001900D928A95E1F70E94750909CFF9
:1016400086E0F801A2E7B2E001900D928A95E1F7F9
:1016500000CFC8010E94B307811175CF8091770236
:10166000816080937702C8010E944507F2CE7A2DEF
:10167000B98AA88A6E2D89890E94C60786E0F6017C
:1016800011928A95E9F7D9CFEE2009F46BCFC80102
:101690000E94B307F82E882309F464CF86E0F8018E
:1016A000A2E7B2E001900D928A95E1F782E792E01D
:1016B0000E9482040E948409C0CF81E08E25D7CE8B
:1016C000ACE0B0E0E6E6FBE00C941D294F835887C0
:1016D00069877A878B879C87CE0107960E94D909F4
:1016E000882369F08A859B85892B39F04F8158853D
:1016F000842F85238F3F09F06BC016E05FC086E022
:10170000FE013796DE01119601900D928A95E1F760
:101710008A859B85892B89F38F81988589238F3FC3
:1017200061F32091410230E0C90101968770992749
:10173000409140024817190671F40E9493071092D5
:1017400041021092400286E0E2E7F2E0DF011D92E2
:101750008A95E9F7D2CF96E0929FD001939FB00D82
:101760001124AE5BBD4FFE01319601900D929A950A
:10177000E1F7809341020E945409BFCF819FC001CD
:1017800011248E5B9D4F0E94D9098823E9F0E091D6
:1017900040021E9FF0011124EE5BFD4F40815181FC
:1017A00062817381848195810E94D007809140027B
:1017B00090E00196877099278093400280914002C3
:1017C000909141028913DACF2C96E3E00C943929E9
:1017D00069857A858B859C850E94D0078ECF682F7E
:1017E00080915F01909160010E9470200895682FA0
:1017F00080915F01909160010E947E200895809108
:101800005F01909160010E948C2008958091980260
:10181000859585958595089580919802877008959E
:1018200090919802977081E009F480E0089580918A
:10183000BB0208959091BB02892B8093BB0208954F
:1018400080959091BB0298239093BB0208951092CB
:10185000BB0208958091BA0208959091BA02892B33
:101860008093BA02089580959091BA02982390933C
:10187000BA0208951092BA020895809199020895CB
:1018800008950E94400C089590912E0392FF08C085
:1018900090919902981721F0809399020E94410C2F
:1018A000089580919902882329F01092990280E08E
:1018B0000E94410C0895CF93DF93E0915F01F09176
:1018C00060018091BB028083E0915F01F091600133
:1018D00080819091BA02892B8083909199029923FB
:1018E00081F0E0915F01F09160018081892B80831C
:1018F00080915F01909160010E94DC1F81110E9424
:10190000510CC0915F01D091600140E250E068E766
:1019100072E0CE010E945E29892B59F080E2FE011F
:10192000A8E7B2E001900D928A95E1F7CE010E94FE
:10193000881FDF91CF91089508950E949C0C08950F
:1019400090912E0392FF11C098E0899F900111247D
:10195000622B609398020E943708809198028595C7
:10196000859585950E949D0C08950E9437080895DD
:101970001092980280E00E949D0C08959091980228
:101980008095892380939802282F277091F4282F1F
:10199000082E000C330B9217130659F090912E036A
:1019A00092FF07C08595859585950E9447080E94FE
:1019B000B80C089590912E0392FB222720F9281746
:1019C00069F080FB92F990932E0380912D03909102
:1019D0002E030E94240D82E00E94BE0C0895809187
:1019E0002E0382FB882780F991E089270E94DA0C78
:1019F000089581E00E94DA0C089580E00E94DA0CDC
:101A0000089590E080E00E94822921E0883E9E4F68
:101A100009F020E0822F089582E090E00E9474296E
:101A2000089583E090E00E9474290895CF9384E0A4
:101A300090E00E947429C82F82E290E00E947429ED
:101A4000982F8C2FCF910895CF93C92F682F84E0C2
:101A500090E00E9488296C2F82E290E00E94882901
:101A6000CF910895AB01BC018FE090E00E949A29CC
:101A70000895AB01BC0183E190E00E949A2908958A
:101A800060E070E0CB010E94390D089560E070E0E5
:101A9000CB010E94320D0E94400D089568EE7EEF4A
:101AA00090E080E00E94A62960E082E090E00E9441
:101AB000882960E083E090E00E94882910923F022C
:101AC00010923E0260E084E090E00E94882964E089
:101AD00082E290E00E94882960E085E090E00E9428
:101AE000882960E086E090E00E9488296FEF87E017
:101AF00090E00E94882940E050E0BA0188E090E040
:101B00000E949A2960E08DE090E00E94882940E0E0
:101B100050E0BA0188E190E00E949A2960E087E1F4
:101B200090E00E94882940E050E0BA018CE190E00A
:101B30000E949A2970E060E080E290E00E94A6296D
:101B400040E050E0BA0188E190E00E949A290E94AA
:101B5000460D08950E944E0D0895682F8EE090E086
:101B60000E94882908950E9454216093C7027093AF
:101B7000C8028093C9029093CA026093C302709313
:101B8000C4028093C5029093C60208950E94542116
:101B90006093C7027093C8028093C9029093CA02EF
:101BA0006093BF027093C0028093C1029093C202FF
:101BB0000895089508950E94DA0D08950E94AA02DA
:101BC00008958DE690E10E94711F0E94D90D0E9438
:101BD000DB0D089581E008950E94EA0D08950895AF
:101BE00008950E94EF0D0E94F00D08950E9470105C
:101BF0000E94210408950E943F210E94E8100E9443
:101C0000F60D0E9452190E949A1C0E94DE0D089542
:101C1000AAE0B0E0EEE0FEE00C9419290E94F41076
:101C20001091BE0280E00E94961018132FC00E94EF
:101C300048218C018091BC029091BD0208171907C0
:101C4000A1F08FEF89838A831B820E9448218160E3
:101C5000782F9D838C8349815A816B818D810E946D
:101C60004D041093BD020093BC020E94511F0E94BC
:101C700085190E940B1D81110E94C60D0E94FA1247
:101C80000E9434042A96E7E00C9435298091CB0217
:101C900081FD0E949C100E94EC0DD82E80E00E94D5
:101CA0009610182F8091BE02181721F1E12EE82618
:101CB00000E0FF24F3948E2D8F21B1F0DD20A1F000
:101CC0000E831F8291E0812F8F2109F490E0988785
:101CD0000E9448218160782F9A8789874E815F8191
:101CE00068858A850E944D040F5FFF0C053019F747
:101CF0001093BE020E94B30DB8CFCF93DF930E9422
:101D0000880FEC01811521E5920708F042C081158A
:101D100030E5930708F09FC0883E910530F5803E7E
:101D2000910508F094C0883A910588F4853A9105A8
:101D300008F086C08130910509F489C0009709F444
:101D400086C0049708F083C0D0E0C0E080C08F3B1D
:101D50009105D0F7C85AD0E0CC0FDD1FC654DE4F36
:101D60000990D881C02DD46472C0811540E29407D7
:101D700050F4C11581E0D80708F069C0CD3ED10507
:101D800018F3D06564C081159044F0F2DF70D06A1A
:101D90005EC0811535E5930718F5811544E5940774
:101DA00008F085C0C11583E5D80708F06CC0C115DF
:101DB00022E5D20708F462C0CE018370992721E0A2
:101DC00030E002C0220F331F8A95E2F7C695C69510
:101DD00080E2C89FE0011124C22BD32BDC6837C0FE
:101DE000811539E59307A8F4811548E5940708F0B3
:101DF00063C0C11586E5D80708F0A6CF8C2F0E94D6
:101E00002A10C82FD0E0DC2FCC27CC27DF71D0627E
:101E10001EC081152AE5920708F453C0905681151B
:101E2000904208F091CF8D2F8F710E942A1090E080
:101E3000982F882788279F719C012C2BE901E7CFD9
:101E4000C55AD0E0C851DE4FC881D0E0D064CE0181
:101E5000DF91CF9108958370992721E030E002C08F
:101E6000220F331F8A95E2F7C695C69540E2C49FBC
:101E7000E0011124C22BD32BDD68E9CFDC2FCC2766
:101E8000C16FD06AE4CFCE018370992721E030E0A2
:101E900002C0220F331F8A95E2F7C695C69540E22D
:101EA000C49FE0011124C22BD32BDA68D0CFD82FE6
:101EB000CC27C46FD06ACBCFD82FCC27C06FD06AC5
:101EC000C6CF8F700E942A1034E0D695C7953A95F8
:101ED000E1F7CF709C2FEC01D069B9CF711110C020
:101EE000653070F4E62FF0E095E0899FE00DF11D7C
:101EF0001124EE0FFF1FE455FF4F85919491089533
:101F000080E090E008950E946E0F0E947D0E08957B
:101F100082389105B9F1B0F48133910509F47DC09F
:101F200048F48932910509F46DC08A32910509F4AB
:101F30007BC008958533910509F45FC0893391050D
:101F400009F10895833E9105D9F138F4803E910559
:101F500029F1823E910579F10895863E9105D9F1E6
:101F6000873E910509F43EC0843E910541F52091DC
:101F70002E0321FF24C080912D0384FD19C087EE1C
:101F800090E0089520912D03237009F05AC020910C
:101F90002E0323FF14C089E290E0089520912D03C1
:101FA00020FD38C030912E0330FF09C024FF43C00C
:101FB00090E080E0089520912D0322FDF7CF089551
:101FC00020912D0322FD3AC030912E0330FD39C0FF
:101FD00024FFF5CFEDCF20912D0323FFF0CF24FD7B
:101FE000E7CFCDCF20912D0323FD2EC030912E03BE
:101FF00031FFEECF84EE90E0089520912D0325FF70
:10200000DECFC9CF20912D0325FD21C020912E03C5
:1020100023FFD5CF89E390E0D2CF20912D0326FF77
:10202000CECF8AE290E0089520912D0326FFC7CFFE
:1020300081E390E0089583EE90E0089582EE90E0D1
:10204000089580EE90E0089586EE90E0089585E38F
:1020500090E0089590912D0392FF06C0282F2871DB
:102060002830F9F4877F846093FF06C0282F2871F9
:102070002831F1F4877E846120912E0320FF06C071
:10208000382F38713830D9F4877F816021FF06C03E
:10209000282F28712831D1F4877E816194FD877EB5
:1020A0000895282F24712430F9F68B7F8860DCCFC7
:1020B000282F2471243101F78B7E8861DDCF382FE2
:1020C0003171313019F78E7F8860E0CF282F217170
:1020D000213121F78E7E8861E1CF80E00895089557
:1020E0000E94010D811102C00E94AA0D0E940C0DD8
:1020F0008093CB020E94160D90932E0380932D03A4
:102100000E946F100E94110D90E00E94E8078091DC
:102110003C0290913D020E940608089508950E9495
:102120008E10089508950E9492100895E82FF0E00F
:10213000E05DFC4F808108950895CF93ABEEB1E050
:1021400040EF51E061E070E08D918F3F91F0E82F1A
:10215000E295EF70F0E0C1A18F709B0101C0220FEA
:102160008A95EAF7922F90959C2391A382A1822BC6
:1021700082A34A175B0741F7CF910895CF93DF936E
:10218000AC01A62FB0E085E0689FF0011124E55175
:10219000FE4F75E081E060E091919F3F81F0C92F93
:1021A000C295CF70D0E028A130E09F7002C0359575
:1021B00027959A95E2F7982F20FD90E0692B880FDC
:1021C000715051F7A40FB51F6C93DF91CF91089513
:1021D0000E949D101092300310922F0381E00E9404
:1021E00019110E9467030895A1E0B0E0EAEFF0E161
:1021F0000C941D29198260E0CE0101960E94BE1048
:1022000090912F03898121E0981301C020E0981359
:1022100080932F0341E060E373E08FE293E00E943C
:102220001A11182F0E946A03812F2196E3E00C9463
:1022300039290895CF92DF92EF92FF920F931F9367
:10224000CF936C017B01042F222349F081E080931E
:10225000CE020E9448219093CD028093CC02C0917F
:10226000CE02C1110AC0C0E08C2FCF911F910F91F7
:10227000FF90EF90DF90CF9008958091CC029091E5
:10228000CD020E946021059770F310E0A801B6010D
:10229000C7010E945E29892B41F0A801B601C70140
:1022A0000E946B291092CE02DFCFC0E0FBCF0E94CC
:1022B0005A230E94FB0D0E94672308950E946C23FD
:1022C0000E94080E0E94862308950E94E1200E9429
:1022D00040230E94E10D0E9457110E945E110E944E
:1022E000F10DFBCF8091D50280FF0DC0609166019A
:1022F00070E0660F771F6038710570F56115710524
:1023000069F1862F089581FF07C06091660184E01E
:10231000689FB0011124EFCF6091660182FD0AC071
:102320008091D4028823A9F0209165016091660113
:10233000821710F088E0ECCF869FC001112433E0B3
:10234000880F991F3A95E1F7622F70E00E94A1284B
:10235000D2CF68E070E0D5CF8FE7089581E008958F
:102360008091D50280FF0CC06091620170E075958C
:102370006795759567956115710549F1862F0895E3
:1023800081FF06C06091620170E075956795F3CF9B
:102390006091620182FD0BC09091D3029923A1F05C
:1023A0006091610180916201961738F0682F70E0AA
:1023B0006038710500F38FE70895899FC0011124EB
:1023C00070E00E94A128F4CF61E070E0D7CF81E0F7
:1023D00008958D3E31F40E94721181958093D90247
:1023E00008958E3E19F40E947211F8CF8F3E31F499
:1023F0000E94721181958093D8020895803F19F44C
:102400000E947211F8CF893F29F40E94B011809385
:10241000DA0208958A3F21F40E94B0118195F7CF26
:102420008B3F31F40E94B01181958093DB020895B7
:102430008C3F19F40E94B011F8CF9FE0980F9830AC
:1024400070F4815F990B21E030E001C0220F8A9582
:10245000EAF78091D702822B8093D70208958D3FAF
:1024600031F48091D50281608093D50208958E3F2A
:1024700021F48091D5028260F7CF8F3FB9F7809128
:10248000D5028460F1CF4091D8028D3E59F48091FD
:10249000D90287FF0DC01092D90241110BC01092D2
:1024A000D40208C08E3E81F48091D90218169CF3A4
:1024B000442381F08091DA029091DB02892B09F0AC
:1024C0005AC01092D30208958F3E49F447FFF0CFCF
:1024D0001092D8028091D9028111ECCFE0CF803FD9
:1024E00019F41416ACF3E4CF9091DA02893F29F481
:1024F0001916F4F61092DA02DBCF8A3F19F497FF2F
:10250000D7CFF8CF9091DB028B3F29F497FFD0CF44
:102510001092DB02CDCF8C3F19F41916CCF3C8CF43
:102520009FE0980F983090F4815F990B21E030E0A4
:10253000B90102C0660F771F8A95E2F7CB0180953B
:102540009091D70289238093D702B2CF8D3F31F487
:102550008091D5028E7F8093D502AACF8E3F21F441
:102560008091D5028D7FF7CF8F3F09F0A1CF809169
:10257000D5028B7FF0CF08950E9448219C01909155
:10258000D8028091D902982B21F03093D202209367
:10259000D1029091DA028091DB02982B21F03093E6
:1025A000D0022093CF0286ED92E00E94A21F0895F0
:1025B00086E0E6EDF2E0DF011D928A95E9F71092E0
:1025C000D4021092D3021092D5020895FC018281A8
:1025D00081110EC0838181110BC08481811108C0DB
:1025E00091E08581811101C090E0892F817008956B
:1025F00081E0FCCFA6E0B0E0E0E0F3E10C941D291F
:1026000086E0E6EDF2E0DE01119601900D928A95EA
:10261000E1F71092D8021092D9021092DA021092C9
:10262000DB028B819C81892B89F08091D102909172
:10263000D2020E946021AC019091D4029923C9F189
:10264000809167018417150608F440C08D819E8132
:10265000892B91F08091CF029091D0020E9460214D
:10266000AC019091D302992309F471C08091630168
:102670008417150608F479C0BE016F5F7F4F86EDA1
:1026800092E00E949E20811105C086ED92E00E949A
:10269000E61281110E94BC1286E0FE013196A6ED81
:1026A000B2E001900D928A95E1F72696E3E00C9452
:1026B0003929209168018AE0289F9001112424176C
:1026C000350720F69F5F9093D40202C09F3FD1F759
:1026D0001B81112359F00E9472119FEF11160CF407
:1026E00091E0899F802D11248093D8021C811123B1
:1026F00059F00E9472119FEF11160CF491E0899F1E
:10270000802D11248093D9023091D802332309F40B
:102710009DCF2091D902222309F498CF45EB3403B1
:10272000C0011124992359F09093D80245EB24035A
:1027300090011124332339F03093D90287CF81E0FF
:102740008093D802F3CF81E08093D9027FCF20918C
:1027500064018AE0289F900111242417350708F0AE
:102760008BCF9F5F9093D30202C09F3FD1F71D8113
:10277000112359F00E94B0119FEF11160CF491E053
:10278000899F802D11248093DA021E81112359F034
:102790000E94B0119FEF11160CF491E0899F802DDB
:1027A00011248093DB023091DA02332309F464CFE1
:1027B0002091DB02222309F45FCF45EB3403C001F3
:1027C0001124992359F09093DA0245EB24039001E8
:1027D0001124332339F03093DB024ECF81E0809314
:1027E000DA02F3CF81E08093DB0246CFEF92FF92D3
:1027F0000F931F93CF93DF93EB01E82FD1110EC0FE
:10280000442321F0F0E0E551FE4FE4916E2F7E2F3E
:102810008E2FCDB7DEB7E6E00C9436290D2F10E0F1
:10282000282F30E0442329F025513E4FF90124910F
:1028300030E0F6E0CF9FC0011124EFEFF0E0BF01E0
:102840000E948D28AB018C2F90E0880F991FA5E581
:10285000A49FB001A59F700D1124861B970B982F84
:10286000990F980FBF01601B710B629FD001639F8E
:10287000B00D729FB00D11248B2F9D9FB0011124BC
:10288000672F7727EF01C61BD70BBE01629FE001C0
:10289000639FD00D729FD00D11247F01E91AF108BA
:1028A000E09EB001E19E700DF09E700D1124672F27
:1028B0007727E61BF70BE29F8001E39F100DF29F45
:1028C000100D1124E12F722F4230510599F048F478
:1028D0004115510569F04130510581F0EB2F8D2FE5
:1028E00007C04430510569F080F046305105B1F71A
:1028F0006E2F8FCFE22F7B2F812FFACFE22F7D2FEC
:10290000F7CFEB2F822F712FF3CF7B2F822FED2F5D
:10291000EFCF41E00E94F613089508950E948914B4
:102920000895CF93DF93762FE901682F842F0E94BB
:102930008E14798368838A83DF91CF910895809183
:102940003103982F9E7F29F4817082608093310338
:1029500008958A34E8F381708864F8CF88E090E0C5
:102960000E947C290895CF92DF92EF92FF926B0133
:102970007C010E949F14B701A60188E090E00E94AC
:102980009A29FF90EF90DF90CF900895E1E3F3E074
:1029900083E0808311828FEF82838383148260813E
:1029A0007181828193810E94B314089580913103D3
:1029B00080FF02C08695089580E0089590913503C8
:1029C000933018F49F5F90933503882351F0609102
:1029D00031037091320380913303909134030E944C
:1029E000B314089581E00E94DE1408959091350398
:1029F000992319F0915090933503882351F06091F9
:102A000031037091320380913303909134030E941B
:102A1000B314089581E00E94F614089570E00E94B6
:102A2000F61A089560916D018091310380FF0BC00B
:102A300080916C0123E0829FC00111248A5C9C4F2D
:102A40000E940E15089580916E0190916F0123E010
:102A5000829FF0011124EA5CFC4F891748F711822C
:102A6000108212828F5F3396F8CF9091310390FFDE
:102A70000EC090916E0120916F0133E0939FF001A1
:102A80001124EA5CFC4F921718F00E941215089569
:102A90008183608342839F5F3396F5CFA3E0B0E0EC
:102AA000E4E5F5E10C941E299091310390FF0AC0F2
:102AB0009E012F5F3F4F0E9491144B8169818A8153
:102AC0000E9435152396E2E00C943A29CF93DF93C8
:102AD000EC01EC81F0E0EA51FF4F4491E1E3F3E0D7
:102AE000628181810E944E158C818F5F8C83DF9182
:102AF000CF910895CF93DF93EC01E1E3F3E04381BD
:102B000062818C810E944E158C818F5F8C83DF9156
:102B1000CF910895A3E0B0E0E0E9F5E10C941C2921
:102B20008C018091DC0281110AC09E012F5F3F4F12
:102B30004FEF6FEF0E9491148A818093DC02F801BD
:102B40006481613069F08091DC0240E0662361F0CD
:102B500040E0623011F44091DC0280E060E004C0AB
:102B60006091DC0240E080E00E943515F80184812C
:102B700090E0019663E070E00E94A1288483239690
:102B8000E4E00C943829A3E0B0E0E9ECF5E10C9422
:102B90001729082FD62EE42EC22E9091310390FFD4
:102BA00029C0E92FE695AE2FB0E0A051BE4F8C9121
:102BB0008093E6029E7F923009F59E012F5F3F4F82
:102BC000802F0E9491144B8169818A810E94351562
:102BD00000933203D0923303E0923403CC2051F0BF
:102BE00060913103709132038091330390913403EB
:102BF0000E94B3142396E9E00C943329823019F42F
:102C0000E0903403E5CF863019F400913203E0CF31
:102C10008930D9F38931E1F6E9516E2F6170B62E12
:102C2000E695F0E0EA51FE4F1491F12C60917001AD
:102C3000F61618F00E941215CBCFF19EC001112498
:102C400070E00E948D28802FB11014C0860F209153
:102C50006E01622F6F0D7727771F9B01220F331FA5
:102C6000260F371F2A5C3C4F4E2D6D2D0E9491146C
:102C7000F394DCCF861BEBCFE1E3F3E09181282FC7
:102C80004381628188E0890F0E94C315089581E025
:102C90000E943C160895E1E3F3E09181282F4381DF
:102CA000628188EF890F0E94C315089581E00E9418
:102CB0004B160895E1E3F3E0628121E1620F08F42D
:102CC0006FEF282F438181810E94C315089581E011
:102CD0000E945A160895E1E3F3E0628121E1621B4C
:102CE00008F460E0282F438181810E94C315089574
:102CF00081E00E946B160895E1E3F3E0438121E156
:102D0000420F08F44FEF282F628181810E94C31582
:102D1000089581E00E947C160895E1E3F3E0438189
:102D200021E1421B08F440E0282F628181810E944A
:102D3000C315089581E00E948D16089520E00E9439
:102D4000C31508959091310390FF0FC0253068F4AA
:102D500030E0F901EE0FFF1FE20FF31FEA5CFC4FBA
:102D60008183608342830E9412150895A3E0B0E03E
:102D7000ECEBF6E10C941D29122F9091310390FF9A
:102D80000BC09E012F5F3F4F0E949114212F4B815A
:102D900069818A810E94A2162396E3E00C94392966
:102DA000EF92FF921F93CF93DF93EC0110E0EE249C
:102DB000EA94F12C60917001161770F00E941215C0
:102DC0009A818C8190FF27C08F5F8C83DF91CF9198
:102DD0001F91FF90EF90089520916E01422F410FB7
:102DE0005527551FCA019A01220F331F280F391F7B
:102DF0002A5C3C4F70E0C7010E94A128962F8C816D
:102E00004091340360913303199F800D11240E9477
:102E100091141F5FCFCF8150D8CFB0E0A0E0E3E1A5
:102E2000F7E10C941629FC0182810FEF80FF01E08D
:102E300010E045E0A42E80917001181798F00E94D0
:102E400012158091DE02013009F04FC0811102C0DD
:102E50008091700181508093DE02CDB7DEB7EAE049
:102E60000C943229C0916E01C12ED12CCC0DDD2DD8
:102E7000D11DCE01880F991FC80FD91FCA5CDC4F26
:102E8000198218821A8234E0E32EF12CB12C809141
:102E9000DE028B0D86301CF16A2D0E947F28892F5F
:102EA000082E000C990BC816D90691F480913403B2
:102EB0008E9DA0018F9D500D1124559547955595D8
:102EC00047959E0160913303809132030E949114D3
:102ED000B00EF1E0EF1AF108D1F61F5FACCF87FF1B
:102EE000DFCF90917001890FDBCF90E00196609168
:102EF000700170E00E94A128AECF0F931F93CF9373
:102F0000DF9380916E0190916F0123E0829FF00129
:102F10001124EA5CFC4F891740F1C0E0D3E06091D6
:102F20007001C61740F10E94121520916A0180912C
:102F3000DD02820F8093DD0290916B01920F9093DE
:102F40006B01191654F4082E000C990B4091700176
:102F50004150550B841795071CF0219520936A0169
:102F6000DF91CF911F910F910895118210821282EB
:102F70008F5F3396D0CF0C2F10E070E0C8010E9415
:102F8000A12820916E01820F482F50E02091DD0290
:102F9000022E000C330B02171307BCF020916B01BB
:102FA000022E000C330B201731077CF08D9F90010F
:102FB00011242A5C3C4F409134036091330380918B
:102FC00032030E949114CF5FAACFFA01EE0FFF1FC8
:102FD000E40FF51FEA5CFC4F118210821282F3CFDE
:102FE000B0E0A0E0E6EFF7E10C941429EC014C818D
:102FF000042F10E09801D8010E94E5289B01AC0144
:103000000E94FB284B015C01E0E2F0E0E01BF10BC9
:10301000A5E5B0E0AC019B010E94FB286B017C019F
:103020009F01DF010E94DD289B01AC010E9406295F
:103030009B01AC01280D391D4A1D5B1DC701B6015E
:103040000E94B528F22E822F90E039E23F1520F140
:1030500043E0249F9001112435952795122F109558
:1030600000E085E5E82EEF1880917001081718F14F
:103070000E9412159C8181E0992319F0903219F475
:103080008FEF8093690180916901890F8C83CDB79F
:10309000DEB7ECE00C94302925E530E0B901681B7F
:1030A000790B9B01220F331F260F371F37FFD4CF19
:1030B0002F5F3F4FD1CF8E2D01FD8F2D20916E01BF
:1030C000622F600F7727771F9B01220F331F260F78
:1030D000371F2A5C3C4F412F609133030E949114AB
:1030E0000F5FC2CF0F931F93CF93DF93EC0110E0DC
:1030F00000E0909170019017110609F06CF40E94A5
:1031000012158C8190E00196817099278C83DF9154
:10311000CF911F910F91089520916E01A801420F48
:10312000511D9A01220F331F240F351F2A5C3C4F7B
:103130004C8160913303809132039695901711066C
:1031400051F04CF0442349F0409134030E94911413
:103150000F5F1F4FCECF4423B9F340E0F7CFE1E339
:10316000F3E080818E7F8083608171818281938191
:103170000E94B3141092E7022FEF80E792E02150F3
:1031800080409040E1F700C000000E9412150895B1
:1031900060913103669570E04BE050E081E791E08B
:1031A0000E945129892B19F481E08093E7020E9443
:1031B00048219093E0028093DF02089590913103BB
:1031C00090FF2BC09170811129C0926090933103C0
:1031D000662351F060913103709132038091330383
:1031E000909134030E94B31460913103669570E0AE
:1031F0004BE050E081E791E00E945129892BA9F032
:103200001092E70281E08093E202409134036091E2
:103210003303809132030E949E160895853210F088
:103220009864D4CF880F982BD1CF0E94C818EACFCA
:10323000682F90913103969581E0890F853208F0CF
:1032400081E00E94DE18089581E00E941819089517
:10325000682F9091310396958FEF890F09F484E2DE
:103260000E94DE18089581E00E942819089561E007
:103270000E94DE180895E1E3F3E08081816080839D
:1032800086950E94371908958091310380FF03C00D
:103290000E94AF1808950E943B19089560E00E94B3
:1032A000DE1808958091E50281112EC00E94010D63
:1032B000811104C00E94AA0D0E94C6140E94AE147F
:1032C00060933103709332038093330390933403FC
:1032D0006E7F61F40E94C6140E94AE1460933103A5
:1032E0007093320380933303909334030E949F14AE
:1032F0001092E7028091310380FF03C086950E94FF
:103300004E1981E08093E50208950F931F93CF93A8
:10331000DF938091E7028823B9F18091E602E09182
:103320003103E695E81BE093E102823091F5F0E08D
:10333000EE51FF4FE491CE2FD0E006E615E18091EB
:10334000E202882361F01092E2020E9448219093E9
:10335000E0028093DF021092E4021092E3020E94E6
:103360004821E091DF02F091E0028E1B9F0B8F3F1E
:103370009F4750F4EC0FFD1FF093E002E093DF0253
:103380008FED92E0F8010995DF91CF911F910F9198
:103390000895863049F4F0E0E152FF4FE491CE2FDA
:1033A000D0E00AE715E1CBCF893051F4E695F0E0A3
:1033B000E452FF4FE491CE2FD0E000ED16E1BFCFF5
:1033C0008F3051F4E695F0E0E752FF4FE491CE2FB5
:1033D000D0E00DE017E1B3CF853149F4F0E0EA52D7
:1033E000FF4FE491CE2FD0E00DE717E1A8CFC8E260
:1033F000D0E000EF17E1883109F4A1CF833239F42E
:10340000E4EDF0E0C591D4910AE815E198CFC4EF5E
:10341000D1E002E718E1843209F491CFC0EDD7E0A2
:103420000DE814E18CCFFA01811101C0FB0109956F
:103430000895CF93DF93C82FD62F0E94D6148C17F0
:1034400048F00E94D6148D1728F40E942419DF91A9
:10345000CF9108958C2F0E943719F9CF1F93CF93E6
:10346000DF93EC01FB01128111117EC00E94170C49
:103470008272CD3CFCE5DF0709F49CC008F041C036
:10348000C73CECE5DE0709F481C0D8F4C43C9CE5F8
:10349000D90709F471C030F4C33CDC4509F469C0B4
:1034A00011E062C0C53C9CE5D90709F46AC046E555
:1034B00056E167E476E1C63CDC4591F70E94131AB9
:1034C00053C0CA3CFCE5DF0709F46AC068F4C83C95
:1034D000ECE5DE0709F45FC047E656E168E776E110
:1034E000C93CDC4559F3DCCFCB3C9CE5D90709F45A
:1034F0005CC04AE055E162EF74E1CC3CDC45F1F29E
:10350000CFCFC23DFCE5DF0709F465C098F4CF3C9E
:103510009CE5D90709F457C008F451C0C03DFCE54B
:10352000DF0709F455C0C13DDC4509F0B9CF6EE0B5
:1035300089E04BC0C53D9CE5D90709F452C058F459
:10354000C33DFCE5DF0709F449C0C43DDC4509F093
:10355000A7CF88E135C0C63D9CE5D90709F444C032
:10356000CE35DD4509F09CCF812FDF91CF911F91A2
:1035700008950E944419F8CF43E359E164E279E1E8
:103580009DCF44E259E163E379E198CF47E456E106
:1035900066E576E193CF48E756E167E676E18ECFC0
:1035A0004AE956E169E876E189CF49E856E16AE9F6
:1035B00076E184CF42EF54E16AE075E17FCF81E0AC
:1035C0000E943719D1CF65E082E00E94191ACCCF52
:1035D00068E086E0FACF64E18FE0F7CF67E185E14C
:1035E000F4CF62E289E1F1CF83E2EACF259A45B1D7
:1035F0004F7D55B15062EFB7F8949B01220F331FF6
:10360000260F371F280F391F2817390741F4EFBF3E
:103610008FE594E00197F1F700C000000895DC0108
:103620006D91CD0178E055B9000000C067FF45B944
:10363000660F000000C000C000C045B900C07A9508
:1036400091F7E2CFCF93DF93EC01FB0182818823D6
:1036500009F464C1C430FDE5DF07E0F5CB3F9CE52C
:10366000D90730F49E0122503C4524313105D8F56C
:103670000E94160D90932E0380932D03C231ECE52A
:10368000DE0709F41FC108F06EC0C9308CE5D80709
:1036900009F4F2C008F03FC0C530ECE5DE0709F4DC
:1036A000DBC058F5C3308CE5D80709F4CDC008F06D
:1036B000CFC080912D038160C230DC4509F4AEC0DB
:1036C00080912D0390912E030E94240D0E94930758
:1036D00080E009C0C63AEDE5DE0751F238F4C236A3
:1036E0009DE5D90729F2DF91CF9108959E012E5AC9
:1036F0003D4523303105B8F7BBCF80912D03806263
:10370000C730FCE5DF0709F489C008F4B1C0809137
:103710002D03806483C0CD309CE5D90709F4BAC07D
:1037200070F480912D038E7FCB30FCE5DF0709F428
:1037300075C008F4A7C080912D038D7F6FC0CF3076
:103740009CE5D90709F4B6C008F4A8C0C031FCE56F
:10375000DF0709F4B3C0C131DC4509F0B1CF809176
:103760002D038F7B5BC0C1159DE5D90709F4B4C05B
:1037700098F5CB3FFCE5DF0709F472C0B8F4C4311B
:103780009CE5D90709F4B6C008F4A2C0C531DC45F0
:1037900009F096CF80912D0382FB992790F921E0C3
:1037A000922790FB82F990FB83F938C0CD3F8CE5DE
:1037B000D80709F477C008F457C0CE3FECE5DE0720
:1037C00009F474C080912E038360CF3FDC4509F07B
:1037D00077CF80932E0374CFC2368DE5D80709F4D6
:1037E00096C068F4C230EDE5DE0709F48CC008F439
:1037F00077C0C330DD4509F063CF80E085C0CE3AA5
:103800009DE5D907E9F068F490912D03892F8E7F0B
:1038100090FF8160C63ADD4509F052CF80932D03B9
:103820004FCFCF3A8DE5D80789F1C03BDD4509F090
:1038300047CF90912E03892F877F93FF8860C9CF50
:1038400080912E038860C5CF80912D038260E6CFE2
:1038500080912D038460E2CF80912D038860DECFBC
:1038600080912E038160B5CF80912E038260B1CF0D
:1038700080912D038061D2CF0E94930780912D0308
:103880008068CCCF80912D038C60C8CF80912E03AF
:10389000877F9FCF80912D038B7FC0CF80912D0399
:1038A000877FBCCF80912E038E7F93CF80912E0394
:1038B0008D7F8FCF80912D038F7EB0CF80912D0390
:1038C0008F7DACCF0E94930780912D038F77A6CF79
:1038D00080912D03837FA2CF80912E038C7F79CF9F
:1038E00080912E03982F909591708E7F892B90FB5D
:1038F00081F96FCF0E94930790912D03892F97FB39
:1039000087F980588BCF81E00E94AD0DD9CE909180
:103910002D03892F8F7E94FF806180CF81E0E3CEDD
:103920008FE891E00197F1F700C0000008950E9430
:1039300054020895FF920F931F93CF93DF9385E076
:103940008093ED020AE212E0C5E2D2E0AE01D801B6
:1039500021E030E08D91E82FE295EF70F0E0F1A0EA
:103960008F70B90101C0660F8A95EAF7962F90957E
:103970009F2191A382A1862B82A3FA018191AF019D
:10398000E82FE295EF70F0E0F1A08F70B90101C06F
:10399000660F8A95EAF7962F90959F2191A382A1B1
:1039A000862B82A3F2E0AF32BF07A1F60E94901CE3
:1039B0006091ED0243EF52E0FA018E2F841B8617CF
:1039C00028F0CDB7DEB7E5E00C943729D8012D916A
:1039D0008D01A22FA295AF70B0E090968C9190E0EF
:1039E0002F7002C0959587952A95E2F7817099917D
:1039F000A92FA295AF70B0E090962C9130E09F7007
:103A000002C0359527959A95E2F790E020FD92E067
:103A1000892B8193D2CFB0E0A0E0E1E1FDE10C94ED
:103A20001829F12CE12C82E0C82ED12C8091ED02D6
:103A3000F81630F08E2DCDB7DEB7E8E00C943429BF
:103A40000F2D10E0F801E65DFD4F8081E82FE29533
:103A5000EF70F0E0E0A1F0E08F7002C0F595E7951F
:103A60008A95E2F7E170D801AB5DBD4F2C91A22F92
:103A7000A295AF70B0E090968C9190E02F7002C04C
:103A8000959587952A95E2F780FD40C080E08E2BC2
:103A9000D801AD50BD4FEC919E2F93709817A1F1B6
:103AA000EE0FEE0FE82BEC93EF70F0E0EB5EFD4FC6
:103AB000E801C251DD4F80819881890F888320E021
:103AC00082305CF0F801E851FD4F80818F5F808388
:103AD00060E08F2D0E94971C21E088818F3F5CF46D
:103AE000F801E851FD4F80818150808361E08F2D86
:103AF0000E94971C21E08881082E000C990BB601CA
:103B00000E94A1288883E22AF39490CF82E0BFCF5D
:103B1000CF93DF93EB0186319C4511F50E94170C82
:103B20009A81992399F08A7A91E009F490E0909330
:103B3000F802811109C089E20E94EF0B0E945B0C20
:103B400080E0DF91CF91089585E3F6CF8091F80270
:103B5000811104C089E20E94F70BF0CF85E3FBCF0F
:103B600081E0EFCF0F931F93CF93DF93C42FD22F1A
:103B7000FC0182818823C9F04093FB020E94482106
:103B80009093FA028093F90280E28C0F883040F41F
:103B9000C77081E001C0880FCA95EAF70E94270527
:103BA000DF91CF911F910F9108951091FB02141393
:103BB00032C08091F9029091FA020E946021883C03
:103BC000910548F5C0E2CD0F1D17B9F080E2810FD5
:103BD000883040F4177081E001C0880F1A95EAF729
:103BE0000E942E05C83048F481E09D2F977001C0D7
:103BF000880F9A95EAF70E942705802F0E941E05DC
:103C0000C83070F6D77081E001C0880FDA95EAF706
:103C10000E942E05C5CF80E28C0F883008F6C77051
:103C200081E001C0880FCA95EAF7F2CF0F939C019B
:103C3000CB01243F4CE5340759F1A8F4293DFCE5BC
:103C40003F0701F12A3D4CE53407D1F1283D3C45C1
:103C500091F406E221EE41EE68ED7CE50E94B21D92
:103C600080E00F910895263FFCE53F07E9F0B0F0B2
:103C7000273F3C45F9F0FC018281882339F11092FD
:103C8000FB02EFCF07E225EE45EE69ED7CE5E6CFDE
:103C900006E221EE40EE64EF7CE5E0CF07E225EEA0
:103CA00044EE65EF7CE5DACF06E221EE42EE66EF08
:103CB0007CE5D4CF07E225EE46EE67EF7CE5CECF7C
:103CC00008E221E045EE6AED7CE5C8CF81E0C9CF8E
:103CD000CF93DF93EC01EA85FB85309719F06C8573
:103CE0007D8509958B810E94330C8C810E94200C6C
:103CF0000E945B0C86E0FE0111928A95E9F7DF9144
:103D0000CF910895CF93DF93EC018D8181FD12C097
:103D100082608D838B810E942D0C8C810E941A0CF5
:103D20000E945B0CE885F985309721F06C857D85D4
:103D3000CE0109951092FF021092FE028D8180FD46
:103D400003C0CE010E94681EDF91CF910895CF93EA
:103D5000DF93EC018A81823039F4FB0182810E9479
:103D60002B088D8182608D83DF91CF910895DB01D7
:103D7000FC018281813029F48D919C910E94EC029A
:103D80000895823039F41396ED91FC9114971296B0
:103D90008C9109950895FC018281813029F4FB0101
:103DA000808191810E9402030895FB0122812223D8
:103DB000E1F0E091FE02F091FF023097B1F0E817D8
:103DC000F90799F02EE0E29FF0011124DF01AB5FCB
:103DD000BE4F2C9124602C93E050FF4F9183808341
:103DE000CF010E94821E0E943A0C0895EF92FF922A
:103DF0000F931F93CF93DF938C0197558F3F9105BE
:103E000011F008F041C07801FF248EE0089FF00116
:103E10001124EF01C050DF4FDB0112962C91EB5FB4
:103E2000FE4F808120FB80F98083222399F10E943C
:103E300048219093FD028093FC028A818F5F8A83E0
:103E40000E94170C8B830E942A0C9B81892B8B83E9
:103E50000E943D0C8C83EE81FF81309721F06C85B0
:103E60007D85CE0109958EE08E9DF0018F9DF00D30
:103E70001124E050FF4F858181FF02C010E000E077
